:020000020000FC
:100000000EC0189518951895189518951895189567
:10001000189518951895189518951895189500E045
:1000200010E020E049E147BB13952395203521F4EA
:1000300020E00395037010E0013020F081F00330E0
:10004000B9F421C0137029F0123031F047EF48BBEA
:1000500005C04EEF48BB02C04FEE48BB3DC0412F2C
:10006000447019F047EF48BB02C04EEE48BB34C0A5
:10007000113031F0133021F017704FEF48BB02C040
:1000800046EE48BB29C01E3009F410E0113088F05C
:1000900099F01330A0F0B1F01530B8F0C9F0173076
:1000A000B8F099F0193070F051F01B3028F009F0D9
:1000B0000FC04EEF48BB0EC046EF48BB0BC046EE2C
:1000C00048BB08C047EE48BB05C04FEE48BB02C066
:1000D0004FEF48BB44E000C041E05FE76FEF000036
:0E00E0006A95E9F75A95D1F74A95B9F79DCF81
:00000001FF
